:030000000219FDE5
:03000B000200A848
:03002B000201557A
:03005B000202DBC3
:030073000202C8BE
:1000800002030406080C10182030406080040608A3
:100090000C10182030406080A0C00003070F1F051F
:1000A000050D050205030302C2AFC0D0C0E0206207
:1000B00014E5256009E473E525F4F58AD262D0E001
:1000C000D0D0D2AF3285268AC262E526F4602AD02B
:1000D000E0D0D0C295C294C293D2AF32C295C2943E
:1000E000C293206F0D20650A7405D5E0FDE57BF411
:1000F0005290D0E0D0D0D2AF32758A00C28DD26299
:1001000001F201B7306805206502D29501B7306869
:1001100005206502D29401B7306805206502D293AC
:1001200001B7D29230680A2065077403D5E0FDD28A
:100130009501B7D29130680A2065077403D5E0FDB8
:10014000D29401B7D29030680A2065077403D5E0D5
:10015000FDD29301B7C2AFC2AD53E6EFC0D0C0E04D
:10016000D2D3D2AFC2CEE52A600720744F152A2120
:10017000BC7800790020742EE580307E01F430E7F1
:100180000278FF53DACF207E0343DA20307E034328
:10019000DA10C2D8C271E580307E01F430E702790E
:1001A000FFC3E89970CB306103752A18207403757A
:1001B0002A18885CD270E86003755F0020740DE532
:1001C0002B6004152B21CC43DA01C2D820700241E8
:1001D0003FA85C206102C270207431C3E894F040F3
:1001E0000374F0F8E8C4540F28F87984B703024187
:1001F0000CC313C3138721200802C313200A06C3AC
:10020000C898F8410C28F8500374FFF8C3E89565C6
:100210005003E565F88822E52D54066022206B1F07
:10022000E536C333C333F8E564C313C313F9C39589
:100230002240028922E82522F52250037522FF85FB
:100240002224A824C3E52495614002A8618825E5FD
:100250006670024183C3E8AA669A5003E8FAE4F99B
:10026000EAC333FBE568F45B29400D2567F8E567D1
:1002700060021567400B41830AC3E5679A50020587
:100280006778FF882620CF0AD0E0D0D043E610D28E
:10029000AD32C2CF053A7801E52A60053074021507
:1002A0002AC3E55C94014005755F0041BE7560009E
:1002B000756900E55F2401F55F5003755FFFD0E0CD
:1002C000D0D043E610D2AD32C2AF53E67F7592FA7A
:1002D0007593FFC260759104D2AF32C2AF53E6EF9F
:1002E000C2ADC0D0C0E0C0F0D2D3D2AFA8FBA9FC51
:1002F000C2D8307102614253DACF207E0343DA1054
:10030000307E0343DA20D271E580307E01F420E7AD
:1003100002611988278928A16F53DACF207E034311
:10032000DA20307E0343DA10C2D8C271307402A1E1
:100330005B7800E580307E01F430E702A15B885CE9
:10034000A14353DACF207E0343DA20307E0343DA21
:1003500010C271206102811B53DACF207E0343DA81
:1003600010307E0343DA20C2D8D27188578958C32F
:10037000E89555F8E99556F97B007E087A00C3E8C0
:10038000948CE994005005755B00810D882178A25A
:10039000E6A8216055C3E894C8E994005008E4D267
:1003A000E4FB7A0A61E8C3E89468E994015008E440
:1003B000D2E3FB7A0F61E8C3E894D0E994025008D5
:1003C000E4D2E2FB7A1E61E8C3E894A0E994055008
:1003D00008E4D2E1FB7A3C61E8C3E89498E9940828
:1003E0005008E4D2E0FB7A787E00C3E89559FCE936
:1003F000955AFD30E70AECF42401FCEDF43400FDDD
:10040000755B00C3EC9AED9E5003755B01885989BA
:100410005A8557558558567802A143C3E89527F861
:10042000E99528F9307C02A127307B02A127307A98
:1004300002A120207502813EE9FDE8FC815DE9C34F
:1004400013F9E813F8307902A120E9C313F9E8138E
:10045000F8307802A120E9C313FDE813FC20612CD9
:10046000C3EC941CED940240028174ED701EC3EC49
:0F04700094C850180529E52970021529C3E529FC
:10047F00940A5002A15B755C00D270A15BE5296004
:10048F000215297888E6F97400207F087896B90359
:10049F0002789EE624FAFEE43400FFC3EC9EFCEDE6
:1004AF009FFD9208B90310A2085007207609D27653
:1004BF0081C6307602C276A2085016B9030DECF44D
:1004CF002401FCEDF43400FD0204E078007900A172
:1004DF0027B90315EC33FCED33FDC3EC940AFCEDA7
:1004EF009400FD50047C007D00C3EC94FFED94005C
:1004FF00400678FF7900A127EC8572F0A4C5F0A221
:10050F00F733F87900400302054378FF79000205BD
:10051F0043E9C313F9E813F8307C0EE9600278FF62
:10052F00C3E81338F8E43400F9C3E894FFE9940002
:10053F00400278FF885CD270206102A15B741FF4C7
:10054F00552F4BF52FC274EB7002D274752A1830E9
:10055F007403752A0A306102A16F20740353DAFE07
:10056F00207403752B06D0F0D0E0D0D0D2AD43E687
:10057F001032790102059F790302059F790A02055E
:10058F009F791E02059F796402059F79C802059F16
:10059F007817E4D5E0FDD8FAD9F6227A147B7802E1
:1005AF0005C67A107B8C0205C67A0D7BB40205C690
:1005BF007A0B7BC80205C6E573D5E001227902E408
:1005CF00D291D5E0FDD294D5E0FDC294D5E0FDC225
:1005DF0091D5E0FDE920E002D29530E002D293E51B
:1005EF0073D5E0FDE920E002C29530E002C29374BA
:1005FF0096D5E0FDD9C9EAF8D5E0FDD8FBDBB8D236
:10060F009122C37C007D0075F00005F0EA33FAEB10
:10061F0033FB50F6EB13FBEA13FAC3E9FFE8FEE8EE
:10062F009AF8E99BF95004EFF9EEF8B3EC33FCEDCF
:10063F0033FDD5F0DFEDF9ECF822E889F08A20D20E
:10064F00D4F8A9F07B0030F70B7BFFF42401F8E915
:10065F00F43400F9E88520F0A4ADF0F8E98520F036
:10066F00A4AFF0FEED2EF974003FFA7C04C3EA1339
:10067F00FAE913F9E813F8DCF48BF030F70AE8F431
:10068F002401F8E9F43400F9E889F0C2D4F8A9F0AC
:10069F002222C3E54113F9E54013F8C3E54498F866
:1006AF00E54599F9500CC3E89480E994FF40160290
:1006BF0006D8C3E8947FE9940050030206D8787FE8
:1006CF0079000206D8788079FF8849894A22E5495E
:1006DF002546F8E54A3547F9854A20E4300701F405
:1006EF003548FA30E709C3EA94F04015020716C3FC
:1006FF00EA940F500302071678FF79FF7A0F02076B
:10070F0016780079007AF0C3E5249561500AC37416
:10071F00019524500B020734E54A20E70E020734F7
:10072F00E54A30E706884689478A482278A5E6FADF
:10073F00C3E54933F8E54A33F9D149E930E70BC34B
:10074F00E89480E994FF4013E16EC3E8947FE99445
:10075F00005002E16E787F7900E16E788079FFE8D2
:10076F0020E715C3E52398F84009C3E89401400337
:10077F000207957801020795E8F424012523F84034
:10078F000302079578FF884B2278A6E6FAA847A9B7
:10079F0048D149E930E70CC3E89401E994FF4016CA
:1007AF000207C9C3E894FFE9940050030207C97810
:1007BF00FF79000207C9780179FFE920E715C3E542
:1007CF004B98F84009C3E8940140030207F0780101
:1007DF000207F0E8F42401254BF840030207F078F4
:1007EF00FF88242278FF20692879A1E76023E5415B
:1007FF00601F74FF8541F0848539F0306A0375F00E
:10080F0005A4F8C5F0600278FFC3E895645002A80C
:10081F0064886322C3E5409440E5419401E5635049
:10082F0003140134046002F5632202083C2275E8C8
:10083F0090227883E6FF30EDF9A8BDA9BE0570C3FD
:10084F00E57094084052757000E9FA79A0E76044AA
:10085F00EA7007E571601B020875C3E895716010B7
:0D086F00E5715006600C140208810460F968
:10087C00020881E571F571C3946D401B7561C0C3AD
:10088C0094044013756180C39404400B756140C39C
:10089C009404400375610075BB0622E561F46002A7
:1008AC000561E570B4070375BB1022743279A78714
:1008BC00F0A4C5F0A2F733F8C3E895614002A86133
:1008CC0088228824882588268864227540007541F2
:1008DC00F022C2AF75C820A8CCA9CDAA3A30CF015E
:1008EC000A75C824D2AFAB3BAC3C883B893CC3E80F
:1008FC009BF8E99C206908F930660221EF2149AD8B
:10090C003D8A3DF9EA9DFA600678FF79FF212EAE0B
:10091C003EAF3F8B3E8C3FA83BA93CC3E89EF8E919
:10092C009FF9C3E54113FBE54013FAE82AF540E9CA
:10093C003BF54150067540FF7541FF2196AA40AB2F
:10094C0041AC40AD417E047F02C3EB9404400D1ECC
:10095C001FC3EB94084005206A021E1FC3ED13FD54
:10096C00EC13FCDEF7C3EA9CFAEB9DFBEF6009C3CA
:10097C00E913F9E813F8DFF7EA28FAEB39FB8A40B8
:10098C008B4150067BFF8B408B41C3EB9402500292
:10099C00D2663069047F0321C17892E6FFC3E53744
:1009AC00948240110FC3E53794A040010FC3EF941C
:1009BC000640027F057E02E541C4540FF9E541C4AF
:1009CC0054F0F8E540C4540F28F8C3E89EFAE994B3
:1009DC0000FB4009C3EA9402EB940050047A02E451
:1009EC00FB413BAA40AB41EBC4FEEAC4540F4EFCA6
:1009FC00C3EA9CFAEB9400FBC3E813C313F8EA2890
:100A0C00FAEB3400FB8A408B41C3EB94024002C2E8
:100A1C00667802EBC4FE7B00EAC4540F4EFAC3EABC
:100A2C0098FA4005C3940250027A027892E6FF309D
:100A3C006002413B855192855293D26043E680C35C
:100A4C00E49AF8E49BF930660241C7E8FAE9FBD373
:100A5C00E913FDE813FC88518952C3EF9403603805
:100A6C00EF20E00DE82CF8E93DF9ECFAEDFB020A79
:100A7C0090E828F8E939F9C3E82402F8E93400F9D8
:100A8C007AFE7BFFC3EF9403400E8A538B54884D40
:100A9C00894E8C4F8D5041FB885389548A4D8B4E17
:100AAC008C4F8D503069127553F07554FF754FF0A3
:100ABC007550FF7551F07552FF41FBE8FAD3E813FE
:100ACC00FC8851C3EF94036020EF20E007E82CF87A
:100ADC00ECFA41E7E8282402F87AFEC3EF940340CD
:100AEC00088A53884D8C4F41FB88538A4D8C4FE5B7
:100AFC0068C3335002646BF568306002610575346D
:100B0C0002D26043E680E52D54066034A840A9412A
:100B1C00C3E913F9E813F8C3E913F9E813F83069DA
:100B2C0004E92440F9C2AF53E67F759100C3E49801
:100B3C00F594E499F595759104D26043E680D2AFB3
:100B4C0022D264754300752000306C03752040027E
:100B5C000B6CD264754300752040306C037520001B
:100B6C0078017901206620E52D54066002C2647973
:100B7C0014E541C313700104F8C3941440027814B3
:100B8C00306904781B791B206010E543600C3069D8
:100B9C0003D53404D26D8116710D0543E59B544089
:100BAC00B52002810030690908C3E8994001186139
:100BBC009320640A08C3E8994002616C6193C26493
:100BCC00C2AF53E67F75910030661275940075952F
:100BDC00F8759104D26043E680D2AF616CE5417E3A
:100BEC00FFC3334005C3334001FEC3E49E7594003C
:100BFC00F59561DDC3E53394015002616C306402FC
:100C0C00616CD80281146193C26DC2AF53E67F75DB
:100C1C009100855394855495759104854D92854E1C
:100C2C0093D26043E680D2AFE52D54066008206A6B
:100C3C00020533020C52306D0D206C0A206407152E
:100C4C008115810215182278003064027801E5378D
:100C5C0075F007A4F9E5F028F5F0E9A2F013A2F17C
:0F0C6C0013A2F213F537C394785003753778C38A
:100C7B00E53795384008D265C295C294C29330606F
:100C8B00028189854F92855093D26043E680222062
:100C9B007D16C2AF754202D291C292306202D293DC
:100CAB00D2AF759F11020E8AC2AF754202D291C2AA
:100CBB0090306202D295D2AF759F11020E8A3072BC
:100CCB0043207D20C2AF754203900133757B02C276
:100CDB0093D290306204D29481E7C291D2AF759FC8
:100CEB0001020E8AC2AF754203900133757B02C2BB
:100CFB0095D292306204D294A107C291D2AF759F64
:100D0B0021020E8A207D17C2AF75420390010EC2DD
:100D1B0093306202D294D2AF759F01020E8AC2AF9A
:100D2B0075420390010EC295306202D294D2AF7518
:100D3B009F21020E8A207D16C2AF754204D292C249
:100D4B0090306202D294D2AF759F21020E8AC2AF4D
:100D5B00754204D290C292306202D294D2AF759F88
:100D6B0001020E8A307243207D20C2AF754205907E
:100D7B000122757B04C294D291306204D295A18D6D
:100D8B00C292D2AF759F11020E8AC2AF7542059007
:100D9B000144757B01C294D291306204D293A1AD10
:100DAB00C290D2AF759F11020E8A207D17C2AF750C
:100DBB004205900104C294306202D295D2AF759F66
:100DCB0011020E8AC2AF754205900118C2943062AF
:100DDB00EBD293D2AF759F11020E8A207D16C2AF54
:100DEB00754206D290C291306202D295D2AF759FF6
:100DFB0001020E8AC2AF754206D292C291306202D4
:100E0B00D293D2AF759F21020E8A307244207D207F
:100E1B00C2AF754201900144757B01C295D29230ED
:100E2B006204D293C133C290D2AF759F21020E8A56
:100E3B00C2AF754201900122757B04C293D29030F0
:100E4B006205D295020E54C292D2AF759F01020E6B
:100E5B008A207D17C2AF754201900118C29530628E
:100E6B0002D293D2AF759F21020E8AC2AF75420197
:100E7B00900104C293306202D295D2AF759F01C22A
:100E8B006522900102757B00C295C294C293D292E7
:100E9B00D291D290C26222788076FF0876FF0876D4
:100EAB00FF0876FF08760308760408760A087601B1
:100EBB00087601087601788C76010876FF0876FFB4
:100ECB000876FF0876FF0876FF0876030876FF089A
:100EDB0076FF0876FF0876250876D00876FA08762E
:100EEB00FA0876040876FF08760108760008767A09
:100EFB000876FF0876010876010876000876030865
:100F0B007600227887E6FFC2727888E6C394036086
:100F1B0008C27DE630E102D27DC27E7889E630E1FF
:100F2B0002D27EC3EF94026008758E01D273020F5A
:100F3B0041758E00C273227880E6149000809378FE
:100F4B00A5F67881E6149000809378A6F67886E66D
:100F5B001490008D9378A7F67886E6F539C3940242
:100F6B005003753902789CE67538FFB40203753867
:100F7B00A0B4030375388278A3E61490009A93F516
:100F8B0066D18D22227896E6FA7897E6FB7888E68A
:100F9B00B40305C3EB940EFB307F047A007BFFC3D5
:100FAB00EB9AFCC3948250027C827572000572EC42
:100FBB008572F0A4C3E5F0947D40F222D27FF190CC
:100FCB001205901205907A007B007C10120586E5C5
:100FDB005C2AFA74003BFBDCF37C04C3EB13FBEAE7
:100FEB0013FADCF7FEC27FF19022757C00757D0051
:100FFB00E5EF20E6037520000520903FFFE5201468
:10100B006006901DFF1460009304600375EF165388
:10101B00D9BF7581C043FF8012058175EF0643B2BE
:10102B0003E5B3240220E70DF521E5E320E0068577
:10103B0021B343E301120E8D7580FF75A40075F18A
:10104B009075D47F75908775A5BF75F2BF75D50068
:10105B0075A60175E241120E8DE4F8F6D8FD7568A0
:0E106B0001120EA21215697898867375300175
:10107900C2AF12059A1205AA1205901205B11205FE
:10108900901205B812059012169212059A12059A35
:10109900120595C2AF757C00757D0078FA79FA3032
:1010A9008707D9FBD8F7021C00120F0E120F421244
:1010B9000F8F120F9078988673120E8D75881075A0
:1010C900890275C82475910475D84075A82275B828
:1010D9000275E690759B80759D0075D10E75BC589B
:1010E90075BB0675BA1175E880120581D2AF120871
:1010F9003975360053DACF207E0343DA20307E0378
:1011090043DA1043DA01C2D8C27112059AD2617B5F
:10111900037A0CE55B70077A0CDB0302109C12055D
:101129009020700302109CC270E55CC3940240E1F8
:10113900E52F541F855E5DF55EB55DD5DAD5C261D3
:1011490053DACF207E0343DA20307E0343DA10C21C
:10115900D8C27178A2E67008D274E52F54E0F52F51
:10116900C275752900120595307409C3E529940AD9
:101179004002D27512058678023074027800C3E500
:101189005C9840F0C2AF1205AA1205AA1205AAD2AC
:10119900AF12059A754C007888E6B40302419C1297
:1011A9000586788CE6C39401500302129CE530C38E
:1011B9009401500302129C757CA5757DF12074354C
:1011C900C3E55C94FF500302129CC2AF1205BFD263
:1011D900AF120595C3E55C940150EFC2AF1205AAA1
:1011E90012058B1205AAD2AF120595C3E55C94FFCF
:1011F90040E90217177F05D27F120F90120595C299
:10120900AFC27F120F90AE5CC3E55C947FD2AF5042
:101219000241AC120581C2AF1205BFD2AFDFD812AD
:101229000FC7C3EE94057897F612059A12169A7F9E
:101239000AD27F120F90120595C2AFC27F120F908A
:10124900AE5CC3E55C947FD2AF50E4120581C2AFB6
:101259001205AA12058B1205AAD2AFDFD4120FC745
:10126900EE24037896F6F87997E7C39482400398B9
:101279005006E824827897F612059A1215B71216C5
:10128900C9120595120F90C3E55C94FF500221C065
:10129900021717757C00757D00C3E55C954C40030A
:1012A900855C4C12059578017988E7B403027805C5
:1012B900C3E55C98400221A0C2AF1205BF1205BF69
:1012C9001205BFD2AF12059A753000E4F531F53237
:1012D9000531E531F4703F0532789AE678191460E2
:1012E90012783214600D787D14600878FA1460035E
:1012F900753200C3E53298401D120E8D1205811515
:101309003275310078998673C2AF1205BFD2AF78B2
:1013190098867312059512058BE52A7005307402BB
:10132900019C78012074027806C3E55C9840A17895
:1013390088E6C394036003120595E52A7003021039
:101349009CC2AF120E8DE4F522F523F524F525F59F
:1013590026F567D2AF7885E6C333F565E4F544F53C
:1013690045F546F547F548F570F52CF52DF5377532
:10137900700875BB1012058112083D30EDFDA8BD3E
:10138900A9BEE97001F8887112084175700875BB2A
:1013990010120F0EC2AF7561FF1208B78522618561
:1013A9002262852263D2AF75220175240175250158
:1013B900752601856069756A017888E6B40307C2F4
:1013C9007D307602D27DD268D269753300120DE67E
:1013D900120E151208D71208DE1208D71208DE12EB
:1013E90008D7120B5E1206A0120C53120C9A12089F
:1013F900DE120B4D306E031206A12066031207F3AD
:10140900306603120823120C53120CC91208DE129B
:101419000B5E306E031206DD120C53120D401208DA
:10142900DE120B4D306E0312073B120C53120D6F77
:101439001208DE120B5E306E03120798120C53125B
:101449000DE61208DE12083D120B4D120C53120E56
:10145900151208411208DE30692F856461856462BE
:0E146900856069756A0179187A0CC3E53399BC
:10147700400CC269D26A8A357561FF021492C3E5CE
:101487005C940140030213EB021520306A25206C9F
:1014970022E535147006C26AD26B61EBF535C3E5F8
:1014A7005C940140030213EB7888E6C3940360035E
:1014B700021520753600788279A4E760027803C3A5
:1014C700E55F985054307404E52A604D7888E6B497
:1014D7000317207D0520760781F030760281F02002
:1014E7006C07D26C856461812A78F0306C0585645D
:1014F700617820C3E54198500261EB306C1BC26CE8
:10150700C27D307602D27DD26A75351285646161FB
:10151700EB0536E55C6002A123753600C2AF120EFB
:101527008D7887E6FE7602120F0E7887EEF6E4F5E1
:1015370022F523F524F525F526F565752C00752D7F
:1015470000D2AF120595120E8D78A4E66006C292FE
:10155700C291C290307409C3E53694044002019CDD
:1015670041D4901A0D78201215F9E520B45A0CA32E
:101577001215F9E520B4A503021597757CA5757DAD
:10158700F1120EA21215B7757C00757D000215B613
:10159700901A0378807B0A1215F9A308DBF9901AD1
:1015A7000F788C7B191215F9A308DBF9901A2822FA
:1015B700C2AF12163C121619901A00740E1215FEBD
:1015C700A374091215FEA374151215FE901A037859
:1015D700807B0A1215FDA308DBF9901A0F788C7B24
:1015E700191215FDA308DBF912164F12162D901AC2
:1015F7002822E493F622E6438F01538FFDFFC3E5CC
:1016070083941C400122EF857CB7857DB7F0538F0B
:10161700FE22438F02438F01857CB7857DB7901AE1
:101627000DF0538FFC22901A0D745AB1FE901A0ECA
:1016370074A5B1FE227A3079D07820901A40B1F99A
:10164700E520F709A3DAF7227A3079D0901A40E734
:10165700B1FE09A3DAF922AB74A875BB010279843C
:10166700BB02027985BB03027986BB04027992BB70
:1016770005027987BB060279A3BB0702799CBB08E1
:10168700027988BB09027989E8F7227C0512059A55
:10169700DCFB22C2AF1205AA1205B11205B812056A
:1016A700BF12058B1205AA1205B11205B81205BFA4
:1016B70012058B1205AA1205B11205B81205BFD281
:1016C700AF22C2AF1205BF1205B81205B11205AAA3
:1016D70012058B1205BF1205B81205B11205AA1221
:1016E700058B1205BF1205B81205B11205AAD2AFB4
:1016F70022AE74AF75C2AF1205AA1205AA1205AAC7
:1017070012058BDEF21205BF12058BDFF8D2AF226E
:10171700D19AD192D192757401757501757600D100
:10172700F87C05AD5C12059AC3ED955C70F5C3E5D1
:101737005C9401400AC3E55C94FF4032021753D121
:101747005EB1B7D19AC2AF75EF16D192DCD50576E7
:10175700C3E5769403500280C6D1920575E57414EB
:1017670090009F93F808C3E57598500280AED19218
:10177700D1920574C3E574940A5002809C120EA29C
:09178700B1B7C2AF75EF16D192A3
:0319FD00020FF5E1
:101A00000E0915FFFFFFFF03040A0101015AA5019A
:101A1000FFFFFFFFFF03FFFFFF25D0FAFA04FF01DE
:091A2000007AFF0101000300FF40
:101A400023585031384123202020202020202020DE
:101A500023424C48454C4923463333302320202031
:101A60002020202020202020202020202020202076
:101C0000C2AFC2D353D9BF7581C043B20343FF8073
:101C1000752438752503B1DC7529A5752AF175E29F
:101C20004043F18053A47F75D4FFD2877DFA7803B7
:101C300079E67C10752200752300901DE97B0675FE
:101C400024987525013087028145208708D8FBD963
:101C5000F9DCF781B7308708D8FBD9F9DCF781B711
:101C6000B19CE493A3C39A6004DDC381B7DBDBB10D
:101C70008E6002812E7B08E493FAA3B16FDBF87AC1
:101C800030B16F752200752300B18EEAFCEBFDC305
:101C9000ED94FE400EB18E8A278B28ED30E0048A49
:101CA000828B83B18E7AC270D8C3ED94FE601950D6
:101CB000CEBD002BEC600F7520007521FF7529004B
:101CC000752A000200008100A827A9280809D80465
:101CD000D90281DCB192EA89AAF281CE0D81A3C337
:101CE000ED94035053EDA2E092007AC5C3E58294CF
:101CF00000E583941C508A200010438F02438F011B
:101D00008529B7852AB7F0300029A827A92808090E
:101D1000438F01538FFDD804D902A133C3E58394C7
:101D20001C4003A3A11689AAE28529B7852AB7F02A
:101D3000A3A116538FFC817F7AC1BD030CE493A34A
:101D4000FAB153DCF8B14B817F8181AA22AB23B178
:101D50006FEBFAEA6222752608C3E52313F523E543
:101D60002213F52250066323A0632201D526EAB18F
:101D7000DCB1DC75260AEAF4200102D287300102C8
:101D8000C287B1DCC3134002C201D526EB22B19257
:101D9000EAFB208702A192308702A197752608AE40
:101DA00024AF25C3EF13FFEE13FEB1E0B1DCC3EAAD
:101DB000133087024480FA30E703632201C3E5232E
:101DC00013F523E52213F52250066323A0632201B5
:101DD000D526D9E52265236523F52222AE24AF2539
:101DE0000E0FDEFEDFFCD20122424C48656C6934E6
:071DF000373164F3300601F6
:00000001FF
